:020000020000FC
:020000000EC030
:0200060032C105
:10001C003DC00FEF01BB0FEF02BB00E004BB0CE3D4
:10002C0005BB0FEF07BB0FEF08BB0FE50DBF04E0DF
:10003C000EBF31E024E181E000E000936200009308
:10004C00630000936600009367000FEF009360005D
:10005C000093640000936100009365000AE005BD05
:10006C000AE803BD00E809BF00E007B900E905BFD5
:10007C0000E808B97894F8940BE006B97894889560
:10008C00FACF0BE806B978948895089504B115B1A8
:10009C00400F511F8A9549F480E408D02A9509F441
:1000AC0022E0022F0A95017007B9189500E110E0C3
:1000BC00400F511F56954795569547955695479520
:1000CC005695479556954795BA0120FD01C06BC0D2
:1000DC002330E0F41091610000916000511720F082
:1000EC00151730F0401720F45093610040936000D6
:1000FC001091630000916200151720F0511730F039
:10010C00041720F4509363004093620050E040E0E9
:10011C0003B304FD04C0709161006091600005FDA3
:10012C0004C07091630060916200773018F06E3FEC
:10013C0008F032C0703019F4603009F42DC090E032
:10014C00A0E0B0E0C0E0723020F4713028F0643FE1
:10015C0018F0645F714006C004EF11E0061B170B2A
:10016C00B801C0E8743020F4733030F0683E20F0F1
:10017C00685E7340C395F6CF643618F4713008F49A
:10018C0004C064567040B395F7CF6A3018F06A50CB
:10019C00A395FBCF962F04C09AE0AAE0BAE0C0E08A
:1001AC0060E070E008952330E0F410916500009158
:1001BC006400511720F0151730F0401720F45093BD
:1001CC00650040936400109167000091660015175C
:1001DC0020F0511730F0041720F45093670040932F
:1001EC00660050E040E003B304FD04C0709165006C
:1001FC006091640005FD04C0709167006091660019
:10020C00D0E0E0E0F0E0723020F4713058F0643F60
:10021C0048F07630F8F4753010F06C3DD8F4645F2B
:10022C00714006C004EF11E0061B170BB801F0E893
:10023C00643618F4713008F404C064567040F395B9
:10024C00F7CFF13838F46A3018F06A50E395FBCFE9
:10025C00D62F03C0DAE0EAE0FAE060E070E008953F
:10026C003A9509F439E001D0189500E008BB393013
:10027C0081F03830A1F03730C9F03630E9F0353044
:10028C0029F1343049F1333071F1323091F13130A0
:10029C0099F1092F4ED002BB01E008BB08950A2F3B
:1002AC0048D00F7702BB02E008BB08950B2F41D05A
:1002BC0002BB04E008BB08950C2F003011F039D0BC
:1002CC0001C00FEF02BB08E008BB08950D2F31D021
:1002DC0002BB00E108BB08950E2F2BD00F7702BB99
:1002EC0000E208BB08950F2F24D002BB00E408BB2A
:1002FC00089500E002BB089503B30073003019F0B9
:10030C00003399F414C000E0009362000093630082
:10031C0000936600009367000FEF0093600000935A
:10032C0064000093610000936500F2DE5CDFA9DEDF
:10033C0008950030B1F00130B1F00230B1F003306B
:10034C00B1F00430B1F00530B1F00630B1F0073047
:10035C00B1F00830B1F00930B1F00038B1F007EF6E
:10036C00089500EC089509EF089504EA089500EB50
:10037C00089509E9089502E9089502E8089508EF3F
:0E038C00089500E8089500E908950FEB089524
:00000001FF
